:1000000000040010FD000000D5000000D700000033
:1000100000000000000000000000000000000000E0
:100020000000000000000000000000003D02000091
:1000300000000000000000007D0400000903000033
:10004000D9000000D900000000000000D900000025
:10005000D9000000D90000000000000000000000EE
:10006000D9000000D9000000D9000000D90000002C
:10007000D9000000D900000000000000D9000000F5
:100080000000000000000000000000000000000070
:100090000000000000000000000000000000000060
:1000A000D9000000D9000000D9000000D9000000EC
:1000B000D9000000D9000000D9000000D9000000DC
:1000C000AC09000000000010040000000400001053
:1000D00090020000FEE7FEE7FEE7002310B5934222
:1000E00003D21C585C500433F9E710BD00238B4247
:1000F00003D200221A500433F9E7704710B50C4CB4
:100100000C4B9C4206D220686168A268FFF7E5FFAD
:100110000C34F5E7084B9C4205D220686168FFF774
:10012000E5FF0834F6E700F0ADFB00F0CBFBFEE79F
:10013000C0000000CC000000D400000043013030BB
:10014000010602040A43024330B500021C1C10439E
:100150001A1C20340449950001326850A242F9D19A
:100160009B00C81830BDC04604000010704700292D
:1001700007D08368002B01D08068FAE7816048606F
:100180008B607047002183688B4206D09A6882603A
:100190008A4200D0506059609960181C704783688B
:1001A000002B12D08B420ED14A688B68002A01D0F6
:1001B00088689060002B01D04A685A600023081CB0
:1001C0004B608B6002E09B68EAE7181C7047806810
:1001D00000280FD0037B8B42F9D142688368002A44
:1001E00001D081689160002B01D042685A600023E1
:1001F00043608360704738B50D1C8468A847201E93
:10020000FBD138BD10B50369002B02D00369013B57
:1002100003610369002B0DD1074C011C201C3830F1
:10022000FFF7BDFF011E05D001230373201C103012
:10023000FFF79DFF002010BD840100102F4A506081
:100240002E4A916070460421084202D0EFF30981E2
:1002500001E0EFF308818A69023A1078274A1060BA
:1002600080B484B06F46264B1A68D2B2032A29D0D4
:100270000AD82449012A1FD015D80220DA68107341
:10028000DA685B68136117E0052A28D024D3802A36
:1002900031D11A49C868026882F30988042170467E
:1002A0000843864621E00320DA681073DA6858684C
:1002B0001061DA689B68536180224B6852051343D2
:1002C0004B6018E00421DA681173DA68596811612B
:1002D000DA689B68536108E0DA68052101E00621CD
:1002E000DA681173DA685B6813618021054A490591
:1002F00053680B43536004B080BC70478401001006
:100300008401001000ED00E0144B1A1C90321168BB
:100310000131116010681249884206D9002010602E
:10032000181C8C30026801320260D868026A0132FF
:100330000262DA68126A8A4206D90021DA6811621A
:10034000D968CA690132CA610122802194331A60D6
:10035000044A490553680B435360704784010010F9
:10036000E703000000ED00E0F8B5424C231C943395
:100370001A68002A06D0201C002238303E491A6034
:10038000FFF739FF271C6037381C0421FFF71FFFD8
:10039000051E20D0381C0321FFF719FF061E16D0BA
:1003A00002696B6A9A420FD12A696B69416A271CFC
:1003B0001160426910371A600123381C2B73291C05
:1003C000FFF7D5FE01233373381C311C01E0381CC4
:1003D000291CFFF7CCFE201C05216030FFF7F7FE3B
:1003E000011E0ED0221C8C3203691268201C1A6078
:1003F000221C9032126810305A6001230B73FFF7F1
:10040000B6FE201C06216030FFF7E1FE011E0AD077
:100410000369C2691A60026A5A6001230373201CCF
:100420001030FFF7A4FEE368002B1AD0E368187BB6
:10043000C0B2062814D800F086FA0405090D0D0D87
:100440000D00FEE7201CE168103006E0201CE1688A
:10045000383002E0201CE1686030FFF788FE00E0E1
:10046000FEE7201C1030FFF78DFE002800D0E06072
:10047000F8BDC0468401001005020000EFF30982B8
:10048000203AF0C244464D4656465F46F0C2203AF6
:100490000B49C868026000B5FFF766FF01BC8646DD
:1004A0000749C86802681032F0CAA046A946B24699
:1004B000BB46203AF0CA103282F309887047C04622
:1004C0008401001008B500F08DF9FA21144B890061
:1004D000186800F0FEF9134901384860C020124B3B
:1004E00000061A6A1202120A02431A6200228A6085
:1004F00007320A60DA691202120ADA611A6A120213
:10050000120A1A62196A094A0A40C02109040A43F8
:100510001A628022064B12061A6080DFC046FEE790
:100520000000001010E000E000ED00E0FFFF00FF21
:1005300000E100E0F7B52824194E4443071C009160
:100540000192FFF7FBFD00220121A051A3593519AB
:100550004033A351019B29736A60AA60AB616F624B
:10056000A359104F1A625A63009A59629A63802203
:10057000491852049962DA633B1C88331B68002BCC
:1005800004D1A3592033A351FD6004E0381C291C79
:100590001030FFF7ECFD88373B6801333B60F7BD57
:1005A0001C0200108401001010B5094C201C1030F2
:1005B000FFF7DCFD201C3830FFF7D8FD201C603031
:1005C000FFF7D4FD002003490122FFF7B3FF10BD60
:1005D00084010010E505000000DFC046704701DF20
:1005E000C046704708B5FFF7FAFFFCE702DFC046D8
:1005F000704703DFC046704704DFC046704705DF21
:10060000C0467047F7B540202F4A304BD16F412488
:100610000143D167D16F00180143D16758682C4955
:1006200064420140802059605968C000014359600C
:100630002848294904250860E02040000C50A024E7
:1006400080202406800121580126294321500821B9
:1006500080240527214D22482E60C167D06FE40118
:100660002043D0675A681F4C8A435A605A680A432D
:100670005A601D4B2968186800F02BF927602B6819
:10068000002B1FD0E12105094902281C00F021F9A7
:10069000FF22164B013820621A601868216A1B6815
:1006A0008019DB430193E12389195B0259436843B5
:1006B00000F00FF9019B18180D4B1860A760236814
:1006C0001E432660F7BDC0460480044000800440FD
:1006D000FFFBFFFF0400FFFF00C0004094800440C8
:1006E00004E100E00040064000000010F0800440FB
:1006F000F4800440A02304221B068821002800D097
:100700008A2189015A507047044B9A68520701D5D3
:10071000D86101E0012040427047C04600400640D9
:1007200008B5FFF76FFFFFF73FFF012006491422CE
:10073000FFF700FF022005490A22FFF7FBFEFFF743
:10074000C1FE002008BDC04651070000A5070000FB
:1007500007B5684601A9FFF74CFF019B0020552B08
:1007600002D00120AA2BF4D1FFF7C4FFF1E708B5AE
:100770000120AA21FFF73AFF08BD08B50120552145
:10078000FFF734FF08BD10B5041C2378002B07D0F9
:100790002078FFF7B9FF23789842F9D10134F4E7C4
:1007A00010BD00001FB5002401235C4005D00B489C
:1007B000FFF7E9FFFFF7DBFF04E00948FFF7E3FF7E
:1007C000FFF7DBFFFA204000FFF706FF6846FFF760
:1007D00013FF02A8FFF713FFE6E7C0465609000023
:1007E0006209000070B5234D00206B6ADB051B0F0A
:1007F000013B0E2B02D8204A9B0098580322696ABD
:100800002B6F1C4E13401D4C022B09D093420FD06E
:10081000012B03D1336C1A40022A1DD0184B21E062
:100820001F2319404900023100F053F820601AE0FC
:10083000326C1A40022A0FD011491F23032A0DD00F
:10084000012A03D0B26813405A1C02E0B2681A4071
:1008500001320B1C534305E0002303E0B268134050
:1008600001334B432360A96F206800F032F8206009
:1008700070BDC046008004407009000000000010F8
:10088000001BB7000C490D48CA6F0D4B0243CA67E5
:1008900000221A6401325A640121586C084A084245
:1008A000FAD00020106751670122596F1142FBD026
:1008B000034B9A677047C0460480044080000400E0
:1008C0000080044008B5FFF72BFF08BD03000B4371
:1008D00021D4002931D00122D207030901E0090106
:1008E00012099942FBD9430801E049005208994294
:1008F000FBD900E04908401A07D35241FAD3014618
:100900001046704749084018F7D29218FAD3401899
:10091000014610467047CB0F00D04942021000D567
:100920004042534008B5FFF7D4FF0CBC521000D32F
:100930004042002A00D549421847F446002000F002
:1009400001F8604770478C4671460139095C4900DF
:100950008E44614670474C45445B4F6E205D200DD0
:100960000A004C45445B4F66665D200D0A0000009E
:1009700020A1070000350C00E0C81000C05C150085
:10098000006A180040771B0080841E00C09121007F
:10099000009F240040AC2700E032290020402C00BA
:0C09A000604D2F0000D4300040E1330017
:0409AC00001BB70075
:04000003000000FDFC
:00000001FF
